:100000000C942B030C9463030C9463030C94630310
:100010000C9463030C9463030C9463030C946303C8
:100020000C9463030C9463030C9431180C947317B1
:100030000C94881B0C9463030C9463030C9463036B
:100040000C9463030C9463030C9463030C94630398
:100050000C9463030C943B1B0C9463030C94630398
:100060000C9463030C9463030C9463030C94630378
:100070000C9463030C9463030C9463030C94630368
:100080000C9463030C9463030C9463030C94630358
:100090000C9463030C9463030C9463030C94630348
:1000A0000C9463030C9463030C946303B206260759
:1000B000BA0684068806BE068B06C106CC069606DE
:1000C0001C079A06D0069E06D406FE06A206D8068F
:1000D0000807A806DE06E8068F06C5069206C806CB
:1000E000AD06E306F406140716078006B6062F07CA
:1000F00055075B0749074F07610767076D07250825
:10010000250858085808D208F008F809F809F50831
:1001100069097A097A09EB0DEE0D170E270E2E0EDE
:10012000390ECF0ECF0ECF0ECF0ECF0E3C0E3E0EA1
:10013000430E670E880E8B0E8E0EB00E8515AC1515
:100140005B17AC155B17F8151B165B1711172117FA
:10015000000000000000000000000000000000009F
:10016000000000000000000000000000000000008F
:10017000000000007E0F00D4FFFFFFC700000078E2
:1001800000000000000000002A2B280000000000F2
:100190000000000000000000000000290000000036
:1001A0002C1E3420212224342627252E362D3738A4
:1001B000271E1F202122232425263333362E3738AD
:1001C0001F0405060708090A0B0C0D0E0F1011126B
:1001D000131415161718191A1B1C1D2F3130232D37
:1001E000350405060708090A0B0C0D0E0F10111235
:1001F000131415161718191A1B1C1D2F3130354CE6
:1002000044454255473A2064697361626C65642EC7
:100210000A0044454255473A20656E61626C656448
:100220002E0A005B735D000A002530313662003A09
:10023000200025303258000A722F632030313233CB
:100240003435363738394142434445460A000A00BE
:1002500025303258006C65645F7461736B3A20001E
:100260004F6E6573686F743A206163746976653A9E
:100270002025640A000A002530325820006B657979
:10028000626F6172645F7265706F72743A2000060B
:1002900031FF0974A1010975150026FF009520752D
:1002A0000881020976150026FF0095207508910245
:1002B000C005010902A10185020901A10005091972
:1002C000012908150025019508750181020501091C
:1002D0003009311581257F95027508810609381589
:1002E00081257F950175088106050C0A3802158164
:1002F000257F950175088106C0C005010980A1010F
:10030000850319012AB700150126B700950175105C
:100310008100C0050C0901A101850419012AA00270
:10032000150126A002950175108100C0050109067E
:10033000A1018506050719E029E7150025019508A3
:10034000750181020507190029EF1500250195F0B7
:1003500075018102050819012905950575019102AC
:10036000950175039101C00660FF0961A101096251
:10037000150026FF009520750881020963150026E7
:10038000FF00952075089102C005010906A101052D
:100390000719E029E71500250195087501810295E7
:1003A00001750881010507190029FF150026FF00C6
:1003B000950675088100050819012905950575013F
:1003C0009102950175039101C05B435D005B445D43
:1003D000005B535D005B575D005B525D0009027B73
:1003E00000040100A0FA0904000001030101000952
:1003F00021110100012240000705810308000109C5
:100400000401000203000000092111010001222261
:1004100000070582032000010705030320000109EE
:10042000040200010300000009211101000122B6AD
:1004300000070584032000010904030002030000F3
:100440000009211101000122220007058503200077
:100450000107050503200001120100020000000849
:10046000474C04000100010200010A03410036006C
:10047000350049000000140341006E006F006D005C
:1004800061006C0079004B00420000000403090485
:10049000290A002575002F002575005D28002564B8
:1004A0000020002564002000256400200025640051
:1004B0007C0025303258006D6F7573656B6579204F
:1004C0005B62746E7C782079207620685D28726586
:1004D000702F61636C293A205B0029001E001F0009
:1004E00020002100220023002400250026002700F0
:1004F0002D002E002A00000046002B0014001A00D8
:100500000800150017001C0018000C001200130052
:100510002F003000000031004B00390004001600AD
:10052000070009000A000B000D000E000F00330049
:1005300034000000280000004E00E10000001D0013
:100540001B000600190005001100100036003700DE
:100550003800E500000052004C00E000E300E2003B
:1005600000000000000000002C0000000000E60079
:1005700021520000500051004F00007C3A003B0027
:100580003C003D003E003F0040004100420043006F
:1005900044004500010000000100010001000100CD
:1005A0000100010001000100010001000100010043
:1005B0000100010000000100010001000100010034
:1005C0000100010001000100010001000100010023
:1005D0000100000001000000010001000000010016
:1005E0000100010001000100010001000100010003
:1005F00001000100000001000100010001000100F4
:1006000000000000000000000100000000000100E8
:10061000010000000100010001006164645F6B657E
:10062000795F6269743A2063616E27742061646443
:100630003A20253032580A0064656C5F6B65795F3B
:100640006269743A2063616E27742064656C3A2095
:10065000253032580A0011241FBECFEFDAE0DEBF8A
:10066000CDBF04B603FE18C080917B0290917C023E
:10067000A0917D02B0917E028730904BA740B04B95
:1006800059F410927B0210927C0210927D0210921B
:100690007E02E0E0F8E3099511E0A0E0B1E0E0EDD2
:1006A000F5E402C005900D92A836B107D9F722E013
:1006B000A8E6B1E001C01D92AB37B207E1F70E9496
:1006C0004C0A0C94E6220C940000FF93EF93E09107
:1006D0006801F0916901309709F00995EF91FF9158
:1006E0000895FC018591803011F0EFDFFBCF089574
:1006F000FF27E0E230E247FF0CC0419597FF09C0B9
:10070000EDE26095709580959095611D711D811D3C
:10071000911D27FF02C0219530E350E2AA27660F02
:10072000771F881F991FAA1FA41710F0A41B639599
:100730005A95A9F7AA3008F0A95FA05DAF93F39589
:10074000611571058105910541F7ED3211F4EF93C3
:10075000F395F21718F43F93F395FBCF8F91B5DF24
:10076000FA95E1F70895E991F9918591803021F0AA
:10077000853219F0AADFF9CF089520E0E894559169
:100780005532C1F3503311F4689455915A3348F4FB
:10079000505390F3220F022E220F220F200D250F0F
:1007A000F4CF0EF4219589919991533619F353376B
:1007B00029F1533559F1BC0188279927E8945C3613
:1007C00021F48991999168945591543639F446EF02
:1007D0007EF077FF0DC08FEF9FEF0AC055374AE0DC
:1007E00039F0583540E121F0523642E009F00895E1
:1007F000FF93EF937DDFEF91FF91B7CFFF93EF93DF
:10080000FC0181918030B9F360DFFBCFFF93EF9360
:1008100068DFF1CFDF93CF93CDB7DEB72596A3DFA7
:10082000CF91DF9108950E94C01F2FEF84E39CE0D9
:10083000215080409040E1F700C000009CE088E13A
:100840000FB6F894A895809360000FBE9093600057
:10085000FFCFA7E1B0E0EFE2F4E00C949D224B8BD8
:100860005C8B6D8B7E8B8F8B61111092060286E004
:100870009E01235F3F4FD901E82F1D92EA95E9F7CA
:1008800095E0FE017396D90101900D929A95E1F7DA
:100890009C894E895F897B897D879E876F87598B6D
:1008A000488BF901DE01179601900D928A95E1F7C8
:1008B000CE0107960E94101381113EC086E0FE0112
:1008C0003796DE01119601900D928A95E1F7FF812E
:1008D000E8856A857B856115710531F0EF3F31F45C
:1008E00081E0FF3F19F403C081E001C080E080FD9A
:1008F00023C02091B30130E0C90101968770992788
:100900004091E40150E08417950779F1F983EA8377
:100910007D836C8396E0929FD001939FB00D11244C
:10092000AC54BE4FFE01319601900D929A95E1F7BD
:100930008093B3010E949D1216E08091E401909192
:10094000B3018917F9F0189FC00111248C549E4FF0
:100950000E9410138823B1F08091E40190E0019689
:10096000877099278093E401E8CF0E94C01F1092FE
:10097000B3011092E401EDEAF1E086E0DF011D929F
:100980008A95E9F76796E3E00C94B922ADE0B0E010
:10099000ECECF4E00C948E22FC01808191812381A7
:1009A0003481232B31F09F3F31F491E08F3F19F4D4
:1009B00003C091E001C090E090FD58C57F0185E043
:1009C000DE01199601900D928A95E1F7F7012281D7
:1009D00089859A85222349F00E94C51E182F682F09
:1009E00089859A850E94351F03C00E94011F182F18
:1009F00069857A85812F0E940D108C01F701828113
:100A0000882309F42CC19801225037472031310541
:100A100008F041C18FEF93E00E941F22811129C18C
:100A2000025036E6A32EBB24B394002379F0A11420
:100A3000F4E0BF0609F41DC1C5010E941F22811107
:100A400001C001502FEFA21AB20AEFCFCE010196DA
:100A50002C0188E0F20111928A95E9F72AE0322E02
:100A600085010F5F1F4FC5010E941F2289831A82D3
:100A7000882309F4FEC0813009F041C06501F2E02D
:100A8000CF0ED11CC8010E941F228A83882309F43B
:100A9000F0C09FEF980F933060F423E0A20EB11CDA
:100AA000C6010E941F228B83882309F4E2C01C82A6
:100AB00029C0843031F54E0133E0830E911C02E0F1
:100AC00010E056018FEFA81AB80AC6010E941F2233
:100AD000F40181934F01882309F4CBC08C3741F492
:100AE000E2E0F0E0EC0FFD1FE00FF11F10820AC002
:100AF0000F5F1F4F65010730110519F7BAC0580184
:100B000001C056018201F8012081222309F4A8CFF7
:100B1000213009F04CC08181813049F46801F2E054
:100B2000CF0ED11CF80182810E9400220AC08230BF
:100B300051F46801F2E0CF0ED11CF80182810E94CD
:100B40003C21860189C0833049F46801F2E0CF0E70
:100B5000D11CF80182810E94D820F3CF843019F093
:100B60000F5F1F4F79C0F80122810E5F1F4F80E099
:100B700090E030E0205331092A30310568F4389E86
:100B8000A001399E500D1124C901840F951F0F5FDC
:100B90001F4FF8012081EDCF009709F45DC0EFE908
:100BA000FFE03197F1F700C000000197F5CFE22F89
:100BB000F0E0E058FE4F2490822F8695869586952A
:100BC00090E0FC01E059FE4F64902770712C022EDA
:100BD00002C0759467940A94E2F7F1E06F227724DB
:100BE000FC01E05AFE4F8490912C022E02C0959495
:100BF00087940A94E2F731E083229924FC01E05BB8
:100C0000FE4FC490D12C02C0D594C7942A95E2F728
:100C100081E0C822DD246114710419F081EE0E9484
:100C20003C218114910419F086EE0E943C21822D12
:100C30000E9400228114910419F086EE0E94D820AF
:100C40006114710419F081EE0E94D820C114D104FE
:100C500019F08CE20E9400220F5F1F4F54CF011544
:100C600037E7130709F042C181E00E946D1F0E941F
:100C700097148091E501877009F4F8C3F701828128
:100C8000882309F4F3C380915B0282FFEFC382E003
:100C90000E945512EBC30115F7E71F0711F481E01D
:100CA00005C0013027E7120721F482E00E947A1F75
:100CB000DECFF801E851FC47E730F10508F4E5C064
:100CC000882309F470C110924D02C8019057839790
:100CD00008F013C184E090E00E94272290935B0209
:100CE00080935A02F801E150F047E232F10520F416
:100CF000EA5AFF4F0C94812280915A028160ACC065
:100D000080915B028860B4C080915A028260A4C066
:100D100080915A0220C080915A0288609DC08091C3
:100D20005B021EC080915B028260A2C080915A0269
:100D3000806192C080915A0280628EC080915A0276
:100D400080648AC00E94C01F80915A02806884C05B
:100D500080915A02886084607FC080915B028260CB
:100D6000816086C080915A028E7F76C080915B023E
:100D7000877F7EC080915A028D7F6EC080915A021B
:100D800020C080915A02877F67C080915B021EC09D
:100D900080915B028D7F6CC080915A028F7E5CC017
:100DA00080915A028F7D58C080915A028F7B54C027
:100DB0000E94C01F80915A028F774EC080915A02C4
:100DC000877F8B7F49C080915B028D7F8E7F50C073
:100DD00080915A0282FB222720F991E0922790FB12
:100DE00082F990FB83F938C080915B02982F90952F
:100DF00091708E7F892B90FB81F93AC080915A02C5
:100E000086FB222720F991E0922790FB86F924C0E7
:100E10000E94C01F80915A0287FB222720F991E08F
:100E2000922790FB87F918C061E001C060E08EE076
:100E300090E00E942D221EC080915A0284FB22273E
:100E400020F991E0922790FB84F906C080915A0224
:100E5000982F909590FB80F980935A020BC0809157
:100E60005B0283FB222720F991E0922790FB83F914
:100E700080935B0260915A0270915B0284E090E083
:100E80000E944B220E94C01FF4CEE858FF4F0C94E2
:100E9000812206E221EE41EE6AE17CE723C007E20F
:100EA00025EE45EE6BE17CE71DC006E221EE40EE4B
:100EB00068E17CE717C007E225EE44EE69E17CE7D4
:100EC00011C006E221EE42EE6CE17CE70BC007E2C6
:100ED00025EE46EE6DE17CE705C008E221E045EE37
:100EE0006EE17CE7C7010E94871CC3CE013097E703
:100EF000190709F0DECE82E0B8CE0631ECE71E0716
:100F000009F494C203309CE71907C9F1C0F4013019
:100F1000FCE71F07D1F100F501153CE7130709F0C5
:100F200047C00E94C01FFFEF24E33CE0F150204087
:100F30003040E1F700C000000E94171B9ACE0B352D
:100F40008CE7180761F10C359CE7190701F10A35A8
:100F50001C4771F581E024C080915402982F909530
:100F6000917090FB80F980935402992319F082E1EB
:100F700092E002C080E092E00E9471037ACE6FEFAF
:100F80007FEF80E090E00E944B220E94130480914A
:100F90005B0282FB882780F991E0892701C080E00D
:100FA0000E94721205C00631FCE71F0709F44EC209
:100FB000F701828100811181882349F0C8010E94D4
:100FC000C51ED82E682FC8010E94351F04C0C80155
:100FD0000E94011FD82EB8018D2D0E940D100E9475
:100FE0001B10B82E192F982EF7010281A580A2940C
:100FF0009FE0A9228091E5018770B9F00023A9F054
:10100000812F807F803421F080E28B0D883068F062
:1010100080915B0282FF09C082E00E94551280919C
:10102000E5018770DD24D3948111D12CC12EC294A7
:101030008FE0C8228C2D90E08C30910508F0D8C14B
:10104000FC01E158FF4F0C948122812F807F1F709B
:10105000882311F01295107F0023B9F0112309F4B1
:10106000B5C180E28B0D883010F0911006C09091D0
:101070000702192B1093070205C090910602192B45
:10108000109306020E94C611A1C18B2D0E94D82088
:10109000112309F4ADC180E28B0D883088F19920CD
:1010A00079F11095909106021923109306022BC036
:1010B000812F807F1F70803211F01295107F8B2D51
:1010C000992029F0F1E09F1609F441C04FC08091AA
:1010D0005B0282FD1BC0002369F0112339F090915F
:1010E0000702192B109307020E94C61180E00E948C
:1010F0003C217EC180E00E94D820112309F478C1F0
:10110000812F0E94BF110E94C61172C1002381F07D
:1011100080910802AA2051F021E0A21207C0182BEA
:10112000181709F465C11093080262C1812B16C01B
:10113000A11003C00E94B91131C031E0A31609F417
:1011400057C1812F0E94EF1F0E94B91151C1002386
:1011500041F085E08A1508F44BC1812F0E94F61FEB
:1011600047C194E09A1508F443C118C0002349F020
:10117000AA2099F3F701858180FF28C18F708583AC
:10118000ECCFAA2059F0893309F02FC1FFEF27EEE9
:1011900033E0F15020403040E1F725C1812F0E941B
:1011A000EF1F26C1812F86958695837019F08130B7
:1011B00061F01EC1002321F08B2D912F937002C08E
:1011C00080E090E00E94551C19C1002321F08B2D76
:1011D000912F937002C080E090E00E94301C0EC1FD
:1011E000602F8B2D0E94002009C1812F8370A9F5EB
:1011F000011102C14B2D429546954770440F440F93
:101200008B2D8F7090E09C01042E01C0220F0A9458
:10121000EAF7B4FE08C08FE090E001C0880F4A955D
:10122000EAF7809501C080E016951695137012308C
:1012300069F088F490917501113019F0822B89239F
:1012400002C0922B892B0E94861FD6C0822B9091C0
:1012500075018927F8CF822BF6CF002319F0812F53
:10126000817001C08695882309F4C6C04B2D429534
:1012700046954770440F440F8B2D8F7090E09C0172
:10128000042E01C0220F0A94EAF7B4FE08C08FE0D2
:1012900090E001C0880F4A95EAF7809501C080E090
:1012A000169516951370123059F078F490913D020E
:1012B000113019F0822B892309C0922B892B06C08B
:1012C000822B90913D02892701C0822B0E946A1FC8
:1012D00093C01F70002339F0812F0E947A1F8B2D3D
:1012E0000E94F61F89C08B2D0E94EF1F812F0E9444
:1012F0006D1F82C08B2D92EF991681F1991538F0F0
:10130000E0EF9E1659F0F1EF9F1619F15BC023EF45
:10131000921659F134EF9316C1F054C0002381F0B6
:1013200084E08A1508F464C01F7181E090E0012E0A
:1013300001C0880F0A94EAF790913D02892720C0E6
:1013400095E09A1508F454C0EFCF80915B0282FDBE
:101350001AC0002329F0812F8F7127C00023D9F3F1
:10136000812F8F710E946D1F43C0002341F01F71B8
:1013700081E0012E01C0880F0A94EAF701C080E0E5
:101380000E946A1F35C0002399F01F71812F0E94AF
:101390007A1F80915B0282FF07C0E8E01E9FC001B8
:1013A000112483608093E501812F0E947A1F20C061
:1013B00081E00E945512F1E0FA15D0F482E00E941B
:1013C000551216C0002321F0AA2029F28B2D8FCEB2
:1013D000AA2031F2893349F42FEF37EE83E0215010
:1013E00030408040E1F700C000008B2D0E94D820E3
:1013F00088EF8C0D843010F40E947A1CDD20B1F14E
:101400008091E50180FD32C0F701128285958595B6
:1014100085950E947A1FC7010E94C6048091E5014C
:101420008595859585950E946D1F20C08091070246
:101430008A7A91E009F490E090936A01811112C0D8
:1014400069E28DE891E00E94EA1B09C080916A017F
:1014500081110AC069E28DE891E00E94B11B0E94EF
:10146000C61107CC65E3EDCF65E3F5CF2D96E2E13C
:101470000C94AA228295982F937344E0949F900134
:1014800011248C7C86958695282B822F8575880F54
:101490002A7A2695822B0895AAE2B0E0E2E5FAE0E6
:1014A0000C948E2285B7806885BF85B7806885BF1C
:1014B00084B7877F84BF0FB6F894A89580916000A9
:1014C000886180936000109260000FBE90E080E819
:1014D0000FB6F89480936100909361000FBE82E98B
:1014E00099E190936901809368010E94B7170E9467
:1014F000D6178091E20084608093E2007894809116
:1015000033028823A1F01091E9001F709091EC0044
:10151000892F817090FD80E8182B1092E90080914E
:10152000E80083FD0E94A3141F701093E90082E07D
:1015300084BD93E095BD9AEF97BD80936E000E94A5
:10154000BE1D811102C00E94AE1D09E011E0BEE087
:10155000EB2EB1E0FB2ED8018D918D018F3F11F064
:101560000E94440FE016F106B1F70EE011E0AEE183
:10157000EA2EA1E0FA2EF80181918F018F3F11F040
:101580000E94440FE016F106B1F78AE0E3E8F1E0CB
:10159000DF01282F1D922A95E9F7EBE6F1E0DF0144
:1015A0001D928A95E9F780E090E00E942722873E0D
:1015B0009E4F21F40E94BE1D811161C067EE7EEF37
:1015C00080E090E00E944B2260E082E090E00E9488
:1015D0002D2260E083E090E00E942D2210927501A0
:1015E00060E074E184E090E00E944B2260E086E0DD
:1015F00090E00E942D226FEF87E090E00E942D2264
:1016000040E050E0BA0188E090E00E943F2260E0B4
:101610008DE090E00E942D2240E050E0BA0188E188
:1016200090E00E943F2260E087E190E00E942D223E
:1016300040E050E0BA018CE190E00E943F2260E07F
:1016400070E080E290E00E944B2240E050E0BA015E
:1016500088E190E00E943F2280E00E948F1D0E945E
:10166000AE1D40E050E0BA018FE090E00E943F22C2
:1016700040E050E0BA0183E190E00E943F2282E026
:1016800090E00E941F228093540284E090E00E9428
:10169000272290935B0280935A020E945B0FEFE334
:1016A000FCE93197F1F700C000000E945B0F8091C8
:1016B000830180FF08C06FEF7FEF80E090E00E9421
:1016C0004B220E94171B83E090E00E941F220E9481
:1016D000861F80E091E09093510280935002F2E3E4
:1016E0004F2EF2E05F2E80913302853009F04BC01F
:1016F00083E292E00E94710300E112E180913302E3
:10170000853009F03CC080913302843021F1109281
:10171000550228E130E040E40FB6F894A8952093F4
:1017200060000FBE4093600083B7817F846083BFF9
:1017300083B7816083BF7894889583B78E7F83BF9A
:101740000FB6F894A895809160008861809360003E
:10175000109260000FBE80913202882309F4CECF30
:101760000E945B0FE3E8F1E081919191892B09F0F0
:101770001FC38DE891E08E179F07B1F7BFCF0E947E
:10178000C01F0E947A1C0E945B0FE8E7EE2EE1E08A
:10179000FE2E03E811E022E831E0D801F701419183
:1017A00051918D919D91842795272E173F0719F010
:1017B000892BA9F322C0892B01F50E947C1B7C0197
:1017C0008091760190917701E816F90609F49FC09F
:1017D0008FEF89A38AA31BA20E947C1B8160782FB4
:1017E0009DA38CA349A15AA16BA18DA10E9429049C
:1017F000F0927701E09276018AC08091540281FDD7
:1018000006C073E8672E71E0772E312C43C087E362
:1018100092E00E94710353E8A52E51E0B52EC12C31
:10182000D12C69E2862E62E0962EDF92CF925F92F3
:101830004F920E940A048FE292E00E947103D50148
:101840008C9111966C90B2E0AB0EB11C0E943A0ADA
:10185000782E862D0E943A0A272D30E0322F22273B
:10186000F901E82BCF019F938F939F928F920E9453
:101870000A0487E292E00E947103FFEFCF1ADF0AA9
:101880000FB6F894DEBF0FBECDBF35E0C316D1044E
:1018900061F6B7CFD3018D909D903D01F701A080F7
:1018A000B180A824B924A114B10441F1212CCC2485
:1018B000C394D12CC5018C219D21892BB1F02EA27E
:1018C0003FA221E0C4018C219D21892B09F420E055
:1018D00028A70E947C1B8160782F9AA789A74EA118
:1018E0005FA168A58AA50E9429042394CC0CDD1C65
:1018F000F0E12F12DFCFD7018D929C923394B2E0AA
:10190000EB0EF11CE5E03E12C5CF0E94701B86E095
:10191000E5E4F2E09E012F5F3F4F7901D90101908C
:101920000D928A95E1F710924702109248021092A8
:10193000490210924A028B81811104C08C81882354
:1019400009F453C080914302909144020E94611BAC
:101950009C0190914002992309F449C22531310537
:1019600008F443C09F3F19F09F5F90934002DB80D3
:10197000DD2061F00E94A51E1D1414F491E001C049
:101980009FEF899F802D112480934702DC80DD200A
:1019900061F00E94A51E1D1414F491E001C09FEF98
:1019A000899F802D11248093480230914702332370
:1019B000E1F0209148022223C1F045EB3403C0013D
:1019C0001124992319F09093470203C081E080937A
:1019D000470255EB2503C0011124992319F0909378
:1019E000480203C081E0809348028D81811104C0C8
:1019F0008E81882309F453C0809141029091420264
:101A00000E94611B9C0190913E02992309F4F4C14C
:101A10002135310508F443C09F3F19F09F5F909333
:101A20003E02DD80DD2061F00E94831E1D1414F44F
:101A300091E001C09FEF899F802D1124809349027E
:101A4000DE80DD2061F00E94831E1D1414F491E0FD
:101A500001C09FEF899F802D112480934A0230910D
:101A600049023323E1F020914A022223C1F045EBE1
:101A70003403C0011124992319F09093490203C043
:101A800081E08093490255EB2503C001112499237D
:101A900019F090934A0203C081E080934A0246E025
:101AA00050E0B70185E492E00E94D922892BA9F485
:101AB0008091470281110FC08091480281110BC0B3
:101AC00080914902811107C081E090914A029111F1
:101AD00003C080E001C081E080FD0E94D71D86E048
:101AE000F701A5E4B2E001900D928A95E1F70E941A
:101AF0007A1CD82E80918201D81631F1D0928201C1
:101B00000E94701B8091540282FF1EC080FF04C09F
:101B100085E592E00E9471038091540280FF0CC021
:101B20001F92DF9280E592E09F938F930E940A04B8
:101B30000F900F900F900F908091540280FF04C07F
:101B40008EE492E00E94710380913302843009F0A8
:101B5000CACD83E08093E9008091E80082FFC3CD85
:101B60008091E80085FF21C00E945C1981111BC093
:101B700080E2C82ED12C570109C08091F100D50117
:101B80008D935D01B1E0CB1AD10869F08091E80036
:101B900085FDF3CF8091E8008B778093E8000E9469
:101BA0005C19882399F391E001C090E08091E800EE
:101BB0008B778093E800992309F495CDE9818E2FE6
:101BC00090E0FC013197E331F10508F0E8C0E557FA
:101BD000FF4F0C9481221A828BE053C08A8182309D
:101BE00009F4FCC050F4813009F0D9C00E94701B88
:101BF0009B838C837D836E83D4C0833041F084309B
:101C000009F0CDC01B821C821D821E82CAC0F70152
:101C1000CE010B96D8012C9111963C910E5F1F4F6F
:101C20003283238332968E179F07A1F7BAC08A8129
:101C3000823021F0853009F4B4C0B1C06B817C8161
:101C40008D819E810E9487220E948A1DAAC04C819C
:101C50006B818A810E945C1D9D83C7C02D813E815E
:101C60003227232732274C816B818A810E94001DF5
:101C700098C00E94271D95C080E14EC082E08A83F3
:101C80008AE98B838EC00A811B81102701271027C8
:101C9000AC80B12C6701C8018A599E4F96012E195C
:101CA0003F092A153B0508F07CC00A39B2E01B0742
:101CB00028F40E941F22F601848303C0D6011496E3
:101CC0001C920F5F1F4FBFEFCB1ADB0AE4CF0A81D4
:101CD0001B81102701271027AC80B12C6701C80198
:101CE0008A599E4F96012E193F092A153B0508F087
:101CF00058C00A39E2E01E0728F4D60114966C9108
:101D00000E942D220F5F1F4FBFEFCB1ADB0AE7CFD8
:101D10000E94F01C46C082E08A8343C00A811B8176
:101D2000102701271027AC80B12C6701C8018696C7
:101D300096012E193F092A153B0598F50034E1E07C
:101D40001E0730F40E941F22D60114968C9302C005
:101D5000F60114820F5F1F4FFFEFCF1ADF0AE6CFA5
:101D60000A811B81102701271027AC80B12C670145
:101D7000C801869696012E193F092A153B0588F45D
:101D8000003421E0120728F4D60114966C910E94C9
:101D90002D220F5F1F4FBFEFCB1ADB0AE9CF8FEF6A
:101DA000898340E250E0B70182E00E94A71A9BCCF1
:101DB00009BD19BD09B400FEFDCF8091D8008F7D0B
:101DC0008093D8008091E00082608093E000809151
:101DD000E00081FDFCCF0E94C01F90CC85E290E026
:101DE0000E941F221B821C821D828E83DACF2B3021
:101DF000310508F0B9CDF9CD2B30310508F00ECE04
:101E00004ECE90915A0292FF0DC0282F2871283093
:101E100019F4877F846006C0282F2471243011F4C0
:101E20008B7F886093FF0DC0282F2871283119F40B
:101E3000877E846106C0282F2471243111F48B7EA3
:101E4000886120915B0220FF0DC0382F3871383037
:101E500019F4877F816006C0382F3171313011F459
:101E60008E7F886021FF0DC0282F2871283119F43A
:101E7000877E816106C0282F2171213111F48E7E69
:101E8000886194FD877E0895F894E82FE295EF70BD
:101E9000F0E031A1282F2F7081E090E001C0880F81
:101EA0002A95EAF7982F9095932391A392A1892BD5
:101EB00082A378940895AAE0B0E0E1E6FFE00C94F4
:101EC0009222AE014F5F5F4F7A018AE0FA011192D0
:101ED0008A95E9F709E011E06A019EE0692E91E038
:101EE000792E88248394912CF80180818F3F09F406
:101EF00047C0F894E82FE295EF70F0E021A18F70D1
:101F0000A40102C0440F551F8A95E2F7CA01922F1F
:101F1000982B91A392A18095892382A3789400C0E5
:101F2000EEE0F1E021E030E0A12CB12C41914F3FF7
:101F300089F0A42FA295AF70B0E090968C9190E0BC
:101F40004F7002C0959587954A95E2F780FD02C0D3
:101F5000C90102C080E090E0A82AB92A220F331FED
:101F600051E0EE31F50711F7F80180818F3F11F054
:101F70000E94440FF0EAFA95F1F7F601B182A082CF
:101F80000F5F1F4FF2E0CF0ED11C6016710609F0F3
:101F9000ABCF4AE050E0B7018BE691E00E94D92236
:101FA000892B89F08AE0F701ABE6B1E001900D9250
:101FB0008A95E1F781E080930B020E947C1B90934D
:101FC0000A028093090280910B02811102C080E015
:101FD00020C08091090290910A020E94611B05971E
:101FE000B0F34AE050E06BE671E083E891E00E94D4
:101FF000D922892B59F08AE0EBE6F1E0A3E8B1E0C1
:1020000001900D928A95E1F781E001C080E0109285
:102010000B022A96EEE00C94AE22753048F4603143
:1020200038F4823028F4462F672F0E945C1D0895F3
:1020300080E090E00895CF93DF938238910569F1B5
:10204000B0F48133910509F477C048F489329105E1
:1020500009F469C08A32910509F473C092C08533CE
:10206000910509F45BC089339105B9F08AC0833EBC
:10207000910591F138F4803E9105D1F0823E9105B1
:1020800031F17FC0863E9105D9F1873E9105E9F196
:10209000843E910509F075C028C020915A0220FDA8
:1020A0005BC021FD59C020915B0223FD61C069C066
:1020B00080915A0280FD4AC080915B0280FF4CC033
:1020C00080915A0284FD50C183EE90E04FC180910F
:1020D0005A0282FF3EC0F4CF80915A0282FD39C07D
:1020E00080915B0280FD38C0EBCF80915B0281FF65
:1020F00039C080915A0284FD37C187EE90E036C125
:1021000080915A0283FF2BC0F4CF80915A0283FD45
:1021100026C080915B0281FD25C0EBCF80915A02E1
:1021200085FD26C022C080915A0285FD1EC0809187
:102130005B0283FF1DC00AC080915A0286FD1BC04E
:102140001DC080915A0286FD19C015C089E390E038
:102150000DC182EE90E00AC180EE90E007C186EEEC
:1021600090E004C184EE90E001C185E390E0FEC000
:1021700089E290E0FBC08AE290E0F8C081E390E061
:10218000F5C0EC01811530E5930708F053C08115C7
:1021900060E4960720F0CE019F70906AE7C0803E11
:1021A000910588F58D3C910518F0CE019065DEC053
:1021B000883A9105C0F4853A910550F08C2F855AE4
:1021C000C82FD0E0C25EDE4F888190E09064CEC020
:1021D0008130910509F4C5C008F4C6C0049708F41D
:1021E000C3C0CE01C3C0813C910508F0BDC08C2F97
:1021F000885AC82FD0E0CC0FDD1FCF5DDE4F88811D
:1022000099819464B3C08115904258F08D2F8F71DD
:102210000E94010F282F2F71CE0199279062922BD7
:10222000A5C0C11581E0D807E0F6C83ED10508F089
:102230009BC0D7CFC03692E5D90708F053C0C03451
:1022400022E5D207B8F08C2F8F718695869570E2C3
:10225000879FA00111248C2F837021E030E0B90109
:1022600002C0660F771F8A95E2F7CB019C68842B2A
:10227000952B7CC0C03232E5D30740F08C2F8F7194
:1022800090E0982F8827816F906A70C0C11562E531
:10229000D607B0F08C2F8695869520E2829FA0010C
:1022A00011248C2F837021E030E0B90102C0660F49
:1022B000771F8A95E2F7CB01842B952B9D6856C03A
:1022C0008C2F8F710E94010F95E0D695C7959A9536
:1022D000E1F7CF70D0E0DC2FCC27D0699E01282B0E
:1022E000C90144C0C03A72E5D70708F58C2F8F7139
:1022F000C03892E5D907A8F48695869570E2879F45
:10230000900111248C2F837041E050E0BA0102C08B
:10231000660F771F8A95E2F7CB019A68822B932B81
:1023200025C090E0982F8827846F906A1FC0C03C1A
:1023300022E5D20750F48C2F8F710E94010F8F710C
:1023400090E0982F8827906211C0C03E32E5D307F5
:1023500058F4CE018F719927982F8827806F906A43
:1023600005C081E090E002C080E090E0DF91CF9175
:1023700008958091080281111092080208958095B5
:10238000909107028923809307020895EF92FF92AC
:102390000F931F93CF939091070280910602982B81
:1023A00090938D01809108028823D9F0892B809326
:1023B0008D0180910801882331F080915A0287FFB6
:1023C00002C08EE101C086E0EFE8F1E090E08150CC
:1023D00028F021912223D9F39F5FF9CF91110E9418
:1023E000B91140E250E066EE71E08DE891E00E94A4
:1023F000D922892B09F453C080E2EDE8F1E0A6EE82
:10240000B1E001900D928A95E1F7E0915002F091D0
:102410005102309709F443C080910801882359F094
:1024200080915A0287FF07C080918D0180938E01B1
:1024300086E080938D010280F381E02D8DE891E0AC
:1024400009958091540282FF2AC080FF04C08DE765
:1024500092E00E9471030DE811E0C8E087E7E82EE2
:1024600082E0F82E8091540280FF0CC0F801808138
:102470001F928F93FF92EF920E940A040F900F9089
:102480000F900F90C1500F5F1F4FC111EBCF809184
:10249000540280FF04C085E792E00E947103CF914F
:1024A0001F910F91FF90EF9008952091E501809585
:1024B00082238093E501982F977099F430E0482F9C
:1024C000082E000C550B2417350759F090915B022C
:1024D00092FF07C08595859585950E946D1F109286
:1024E000E5010895CF9390915B0292FB222720F99A
:1024F000281709F1C82F892FC0FB82F980935B024E
:1025000060915A0270915B0284E090E00E944B223D
:1025100082E00E9455128091540280FF0CC01F92ED
:10252000CF9380E692E09F938F930E940A040F90CE
:102530000F900F900F90CF9108958091E4019091AA
:10254000B301891719F08F5F8770FBCF08950F9340
:102550001F93CF93DF938091B20182958F7009F022
:102560005AC08091AF01882309F455C08091E401DD
:102570001091B3016091AD017091AE01C091B001B5
:10258000D091B10191E06F3F09F090E0292F06E072
:10259000811709F440C0209721F07F3F21F030E0FF
:1025A00003C031E001C0322F90E030FD31C0089F00
:1025B000F001099FF00D1124DF01AC54BE4F1196BC
:1025C0003C911197371324C03C91361321C01296C9
:1025D0003C91129731111CC013964D915C91149748
:1025E0004C1B5D0B483C510598F48091B2018F70F3
:1025F00080618093B201E754FE4F80818F708061CB
:1026000080838DEA91E00E94C6040E949D1203C05F
:1026100001968770BDCFDF91CF911F910F910895E3
:10262000A1E1B0E0E6E1F3E10C9495228C0185E0B4
:10263000F801DE011D9601900D928A95E1F7F801EF
:10264000E2809091AD016091AE014091B001509156
:10265000B1014115510531F06F3F31F481E09F3FE9
:1026600019F403C081E001C080E0F82FF1709F2EC3
:1026700080FD1BC1F80130812181C380D4808DEAA7
:10268000A82E81E0B82EF090AF01F601E41BF50B07
:10269000FF2009F4C7C08091B201E83CF10508F0C1
:1026A00092C0482F407F09F051C0621311C09313AC
:1026B0000FC0FE2CE1100CC08F7080618093B201BE
:1026C000C5010E94C6048091B201F80185832AC128
:1026D000C114D10431F02F3F31F481E03F3F19F4B0
:1026E00003C081E001C080E080FD03C081E08E2551
:1026F00002C080E090E0F82FF170FF2E80FF1CC038
:102700008091E4014091B30156E0841709F4E8C0D8
:1027100090E0589FF001599FF00D1124EC54FE4FAA
:102720006181261306C06081631303C06281E612D3
:1027300003C001968770E9CFFE2CEE2009F4F2C0A9
:102740008091B20181608093B20149C0621306C0DA
:10275000931304C0E11002C0F80186C0C8010E94B2
:10276000891F882351F1EE2041F12091B201822F7F
:1027700082958F7090E0029774F08091AD019091F6
:10278000AE0198878F831986DB86CA862C87CE0197
:1027900007960E94C60486E0F801ADEAB1E0019018
:1027A0000D928A95E1F70E94A7120AC06217C9F03C
:1027B000C8010E94891F81111EC0C8010E94C60461
:1027C000FF24F394AFC0482F407F81F78DEA91E05A
:1027D0000E94C60486E0F50111928A95E9F7F12C72
:1027E000A1C09313E5CFE110E3CFF8018583C801C1
:1027F0000E94C60454C0EE2001F32091B201822F42
:1028000082958F7090E0029734F28091AD019091A3
:10281000AE019A8389831B82DD82CC822E83CE0116
:102820000196B7CFE83CF105D0F5FE2CEE2029F259
:10283000621327C0931325C02091B20120FD18C058
:10284000822F82958F70482F50E04115510581F0FD
:10285000F80125834F30510541F08F5F982F9295F5
:10286000907F822F8F70892B8583C8010E94C604B8
:1028700086E0F801ADEAB1E001900D928A95E1F7AA
:1028800051C0C8010E94891F811185CF8091B2017A
:1028900081608093B201C8010E94C60443C086E0F3
:1028A000F50111928A95E9F73DC0EE2009F485CF34
:1028B000C8010E94891FF82E882309F47ECF86E084
:1028C000F801ADEAB1E001900D928A95E1F78091AF
:1028D000AD019091AE010E94F41E0E94A71222C089
:1028E0003D872E878D859E850E94F41E292F229577
:1028F0002F70223028F49F7039F0811105C00BC071
:10290000243028F49F7049F4805E883020F0C8019C
:102910000E94C6049F2CF92C05C0F8019581907F78
:1029200099F7F9CF8F2D6196EBE00C94B12280914D
:102930003D02982F9670963011F4886001C0877F11
:102940000E946A1F0895AAE2B0E0E9EAF4E10C945B
:102950009D22E5E3F2E08091F100819342E0ED33C6
:10296000F407C9F780913602833009F463C030F46C
:10297000813071F0823009F49DC0B4C08A3009F40E
:1029800089C08B3009F46EC0893009F0ABC020C01B
:1029900080913502813A09F0A5C08091E800877FD7
:1029A0008093E8008091390290913A02892B21F4BA
:1029B00060E281E192E003C060E080E090E070E0DE
:1029C0000E94491A8091E8008B778093E8008AC0C2
:1029D00080913502813209F085C080913902909151
:1029E0003A02009719F0029709F07CC08091E80044
:1029F000877F8093E8008091E80082FD05C0809188
:102A000033028111F8CF6EC02091F3008091F20063
:102A100090E0922B029731F48091F100813011F017
:102A2000863021F48091F100809310028091E800BB
:102A30008B7754C080913502813A09F053C0809160
:102A4000390290913A02892B09F04CC08091E8003C
:102A5000877F8093E8008091E80080FFFCCF809121
:102A6000080137C0809135028132E1F58091390249
:102A700090913A02892BB1F58091E800877F80938D
:102A8000E8000E94F51980913702809308010E94A6
:102A9000C01F28C080913502813221F58091E80065
:102AA000877F8093E8000E94F51980913802809317
:102AB0000F0218C080913502813AA1F48091E8009C
:102AC000877F8093E8008091E80080FFFCCF8091B1
:102AD0000F028093F1008091E8008E778093E800E8
:102AE0000E94F5198091E80083FFE5C180913502CD
:102AF00090913602492F50E04A30510508F0DBC171
:102B0000FA01E256FF4F0C948122803821F082387E
:102B100009F0D1C108C0809131029091320299230D
:102B200089F082600FC0809139028F70873008F081
:102B3000C2C18093E9008091EB0085FB882780F972
:102B40001092E9009091E800977F9093E8008093BD
:102B5000F1001092F10071C1282F2D7F09F0ABC157
:102B6000882319F0823061F0A6C18091370281304C
:102B700009F0A1C1933009F080E0809332022EC0A9
:102B80008091370281112AC0809139028F702FEF16
:102B9000280F263008F08FC18093E9002091EB00C8
:102BA00020FF1CC0933021F48091EB00806214C0A0
:102BB0009091EB0090619093EB0021E030E0A9014F
:102BC00002C0440F551F8A95E2F74093EA00109225
:102BD000EA008091EB0088608093EB001092E9009E
:102BE0008091E800877F8093E8000E94F51963C117
:102BF000811161C1109137021F778091E3008078C5
:102C0000812B8093E3008091E800877F8093E80028
:102C10000E94F5198091E80080FFFCCF8091E300CD
:102C200080688093E300111102C082E001C083E05C
:102C30008093330240C18058823008F03CC120911B
:102C40003702309138022C3D53E0350779F583E0A7
:102C50008A838AE289834FB7F894DE01139620E0D5
:102C60003EE051E2E32FF0E050935700E49120FF63
:102C700003C0E295EF703F5FEF708E2F90E0EA3077
:102C800010F0C79601C0C0968D939D932F5F24319D
:102C900049F74FBF8091E800877F8093E8006AE2A0
:102CA00070E0CE0101960E94491AB5C080913902A8
:102CB00090913A02432F552743305105A9F068F40B
:102CC0004130510509F406C14230510509F0F3C005
:102CD0008BE790E0EDEDF3E04BC04132510529F177
:102CE0004232510589F1E7C0C90199278130910528
:102CF000A1F058F0029709F0DEC0EAE6F4E0E491B2
:102D00008E2F90E0EAE6F4E030C0ECE8F4E0E491E5
:102D10008E2F90E0ECE8F4E028C0E6E7F4E0E491E0
:102D20008E2F90E0E6E7F4E020C08430910508F0B3
:102D3000C2C0880F991FFC01E15AFE4F0190F0813B
:102D4000E02D89E090E014C08430910508F0B3C014
:102D5000FC01EE0FFF1FE95AFE4F0190F081E02DBC
:102D6000DC01AD5ABE4F8C9190E0009709F4A3C0EE
:102D70002091E800277F2093E80020913B023091CA
:102D80003C028217930708F49C0140E021153105AD
:102D900089F180913302882309F43DC08530D9F14F
:102DA0008091E80083FD37C08091E80082FD2FC04C
:102DB0008091E80080FFEACF4091F3008091F2001B
:102DC00090E0942B2115310559F08830910540F49D
:102DD00044914093F1003196215031090196F2CF90
:102DE00041E0089709F040E08091E8008E778093F9
:102DF000E800CCCF4111CDCF0AC0809133028823A7
:102E000051F0853041F08091E80083FD04C080914D
:102E1000E80082FFF2CF8091E8008B778093E80092
:102E20004AC0803809F047C08091E800877F8093CE
:102E3000E800809134028093F1008091E8008E7761
:102E4000D2CE811138C080913702909138029927F3
:102E500002978CF58091E800877F8093E8001091BD
:102E60003702109334020E94F519111106C08091A7
:102E7000E30087FD02C081E001C084E0809333025B
:102E800042E061EC81E00E94141A42E261EC84E0CD
:102E90000E94141A42E261EC82E00E94141A42E29B
:102EA00060EC83E00E94141A42E261EC85E00E942B
:102EB000141A809133028091E80083FF10C0809142
:102EC000E800877F8093E8008091EB008062809328
:102ED000EB0005C082E190E0E8E5F4E049CFAA9676
:102EE000E3E00C94B9221F920F920FB60F921124B7
:102EF0002F933F934F935F936F937F938F939F9302
:102F0000AF93BF93CF93DF93EF93FF93C091E9000B
:102F1000CF708091EC00D82FD17080FDD0E8109256
:102F2000E9008091F000877F8093F00078940E9400
:102F3000A3141092E9008091F00088608093F00063
:102F4000CD2BCF70C093E900FF91EF91DF91CF912E
:102F5000BF91AF919F918F917F916F915F914F91B1
:102F60003F912F910F900FBE0F901F901895E8ED95
:102F7000F0E080818E7F80831092E2001092DA0070
:102F80001092E100A0EEB0E08C9181608C93808182
:102F90008F77808319BCA7EDB0E08C918E7F8C93E6
:102FA00080818F7E808310920E020895A0E0B0E0B1
:102FB000ECEDF7E10C949822C8EDD0E088818F7E8B
:102FC0008883E7EDF0E080818160808384E082BFC8
:102FD00081E080930E0288818E7F888302EE10E06C
:102FE000F80110821092DA0081EEC82ED12CF60181
:102FF000108288818F778883888180688883888120
:103000008F7D888319BC1092330210923402109283
:1030100032021092310290EEE92EF12CF7018081FC
:103020008B7F808388818160888342E060E080E0DC
:103030000E94141AF60180818E7F8083F8018081BE
:1030400081608083808188608083F70180818E7FAA
:103050008083888180618883CDB7DEB7E8E00C94F7
:10306000B4221F920F920FB60F9211242F933F9309
:103070004F935F936F937F938F939F93AF93BF9380
:10308000EF93FF938091E10082FF49C08091E200BD
:1030900082FF45C08091E1008B7F8093E100209109
:1030A0000D022F5F822F62E30E946122992319F0A3
:1030B00020930D0234C010920D0280910C028823DF
:1030C00071F180913302843041F58091E9008F7075
:1030D0002091EC00922F917020FD90E8892B95E0D3
:1030E0009093E9009091EB0090FF14C09091EE0056
:1030F00097FF10C09091E80095FF03C01092F10077
:10310000F9CF9091E80090FF05C09091E8009E777C
:103110009093E8008F708093E90010920C028091E8
:10312000DA0080FF32C08091D80080FF2EC08091ED
:10313000DA008E7F8093DA008091D90080FF1CC076
:1031400080E189BD82E189BD09B400FEFDCF81E047
:103150008093330289EC93E00E94710380910E0208
:10316000811113C00E94B7170E94D6178091E20008
:1031700084608093E20009C019BC109233028DEC88
:1031800093E00E94710310920E028091E10080FF93
:103190001BC08091E20080FF17C08091E2008E7F0B
:1031A0008093E2008091E20080618093E200809150
:1031B000D80080628093D80019BC85E080933302E8
:1031C00081ED93E00E9471038091E10084FF34C09F
:1031D0008091E20084FF30C080E189BD82E189BD39
:1031E00009B400FEFDCF8091D8008F7D8093D80078
:1031F0008091E1008F7E8093E1008091E2008F7EDC
:103200008093E2008091E20081608093E2008091EF
:103210003402882311F084E007C08091E30087FD29
:1032200002C081E001C083E08093330285ED93E02A
:103230000E947103809133028091E10083FF2BC0D3
:103240008091E20083FF27C08091E100877F809317
:10325000E10082E080933302109234028091E10019
:103260008E7F8093E1008091E2008E7F8093E20068
:103270008091E20080618093E20042E060E080E0C3
:103280000E94141A8091F00088608093F00089ED0C
:1032900093E00E947103FF91EF91BF91AF919F91D5
:1032A0008F917F916F915F914F913F912F910F90EF
:1032B0000FBE0F901F9018952091E4003091E5000B
:1032C00095E64091EC00842F817040FF23C08091EF
:1032D000E80080FD1DC080913302882399F085307D
:1032E00099F08091EB0085FD11C04091E400509170
:1032F000E5002417350729F3915011F09A01E1CF29
:1033000084E0089582E0089583E0089581E00895BF
:1033100080E008954091E80042FFDDCF089580915C
:10332000100208959FB7F89410920C029FBF9091DD
:103330003302943009F057C09091E9009F703091AA
:10334000EC00232F217030FD20E8922B25E0209304
:10335000E9002091EB0020FF43C02091EE0027FF01
:103360003FC020915C02222321F02091E80025FF3C
:1033700037C010925C0226E03091E80035FD15C0A0
:1033800030913302343061F53091EB0035FD28C0C7
:10339000215021F481E080935C0222C0EFE9FFE03C
:1033A0003197F1F700C00000E7CF8093F1008091E2
:1033B000E80085FD0AC08091E80080FFFCCF809185
:1033C000E8008E778093E80006C08FB7F89421E07C
:1033D00020930C028FBF9F709093E90080E00895C6
:1033E0009F709093E9008FEF08958091350287FFD9
:1033F00011C08091E80082FD05C0809133028111E7
:10340000F8CF11C08091E8008B770BC08091330218
:10341000882349F08091E80080FFF8CF8091E80090
:103420008E778093E8000895982F973068F59093F1
:10343000E900981739F07091EC002091ED0050915F
:10344000F00003C0242F762F50E021FD02C09F5FC3
:10345000ECCF3091EB003E7F3093EB003091ED00EC
:103460003D7F3093ED003091EB0031603093EB0005
:103470007093EC002093ED005093F0002091EE004B
:1034800027FDE5CF80E008958F708093E90081E00B
:10349000089520913B0230913C022617370748F0EF
:1034A0006115710539F42091E8002E772093E8002A
:1034B00001C0B901FC0120E06115710579F180912D
:1034C00033028823F1F18530F1F18091E80083FD2A
:1034D0003CC08091E80082FD2EC08091E80080FF12
:1034E000EBCF2091F3008091F20090E0922B6115D8
:1034F000710551F08830910538F421912093F10045
:10350000615071090196F3CF21E0089709F020E09E
:103510008091E8008E778093E800CECF2111CFCF45
:103520000AC080913302882361F0853061F0809178
:10353000E80083FD0AC08091E80082FFF2CF80E0BE
:10354000089582E0089583E0089581E008950F933F
:103550001F93CF93DF938B01EA0190913302943054
:1035600079F58F708093E9008FEF9091E80081509A
:1035700095FD06C095ED9A95F1F700008111F5CF04
:103580008091E80085FF1CC00E945C19882361F0CF
:103590008091E8008E778093E80012C0F801819155
:1035A0008F018093F1002197209791F38091E8009B
:1035B00085FDF4CF8091E8008E778093E800E4CF1A
:1035C000DF91CF911F910F91089543E050E0BC012E
:1035D00084E00E94A71A089546E050E0BC0184E010
:1035E0000E94A71A0895CF93DF93EC018091080100
:1035F000811105C048E050E0BE0181E00BC0809120
:103600005A0287FF03C040E284E002C048E081E044
:1036100050E0BE010E94A71A80E2FE01A1E1B2E0E3
:1036200001900D928A95E1F7DF91CF91089581E0A5
:103630008093E00080E28093D8001092C9008FE16F
:103640009EE40197F1F700C0000087E090EBDC01F9
:1036500080937B0290937C02A0937D02B0937E02C4
:103660009CE088E10FB6F894A895809360000FBEA7
:1036700090936000FFCF78941F920F920FB60F9235
:1036800011248F939F93AF93BF9380915602909193
:103690005702A0915802B09159020196A11DB11D87
:1036A0008093560290935702A0935802B093590208
:1036B000BF91AF919F918F910F900FBE0F901F9070
:1036C00018959C014FB7F89480915602909157023B
:1036D000A0915802B09159024FBF821B930B0895DD
:1036E0002FB7F8946091560270915702809158025A
:1036F000909159022FBF08952FB7F89480915602E8
:1037000090915702A0915802B09159022FBF08958D
:103710001F920F920FB60F9211248F939F93AF9326
:10372000BF9380915502811113C0809156029091F0
:103730005702A0915802B09159024196A11DB11DA6
:103740008093560290935702A0935802B093590267
:10375000BF91AF919F918F910F900FBE0F901F90CF
:10376000189520910801222351F120915A0227FF38
:1037700026C0262F2695269526952E3178F4FC0115
:10378000E20FF11D677081E090E001C0880F6A953B
:10379000EAF780959281892382830895809154026B
:1037A00080FF17C01F926F9388E396E09F938F93DB
:1037B0000E940A040F900F900F900F900895FC0143
:1037C00006962281621301C012823196E817F9072A
:1037D000C1F7089520910801222349F120915A024E
:1037E00027FF25C0262F2695269526952E3170F485
:1037F000FC01E20FF11D677081E090E001C0880FCD
:103800006A95EAF79281892B828308958091540208
:1038100080FF25C01F926F938AE196E09F938F935C
:103820000E940A040F900F900F900F900895FC01D2
:1038300032962FEF30E04191641789F02F3F19F451
:10384000411101C0232F3F5F3630A9F72F3F39F0D8
:10385000FC01E20FF11D27FDFA956283089508959A
:10386000A3E0B0E0E6E3FCE10C949E22209152023A
:103870003091530228173907A1F090935302809397
:103880005202E0915002F0915102309751F024E041
:1038900029839B838A830680F781E02DCE010196E0
:1038A00009952396E2E00C94BA22A3E0B0E0EBE5A0
:1038B000FCE10C949E2220914E0230914F02281779
:1038C0003907A1F090934F0280934E02E09150028D
:1038D000F0915102309751F023E029839B838A8332
:1038E0000680F781E02DCE01019609952396E2E04E
:1038F0000C94BA22E0915002F0915102309729F0D5
:103900000190F081E02D0995089580E008950F93CE
:103910001F93CF93DF93C42FD22FFC018281882382
:10392000B1F040934D020E947C1B90934C02809317
:103930004B0280E28C0F883008F04DC0C77081E0E8
:1039400001C0880FCA95EAF70E94F61F44C0809113
:103950004D02481330C080914B0290914C020E945E
:10396000611B883C910538F510E21D0FCD17B9F0A9
:1039700080E28C0F883040F4C77081E001C0880F6E
:10398000CA95EAF70E94EF1F183010F581E09D2FCD
:10399000977001C0880F9A95EAF70E94F61F802F52
:1039A0000E9400221830B8F4D77081E001C0880F5F
:1039B000DA95EAF70AC080E28C0F883060F4C770AD
:1039C00081E001C0880FCA95EAF70E94EF1F03C08B
:1039D000802F0E940022DF91CF911F910F910895B7
:1039E000CF93DF93C6E6D1E060E0CE010E942D22A6
:1039F0002196C11584E0D807B9F7DF91CF910895DA
:103A00001F93CF93DF93962F8230E8F46530D8F47C
:103A10004031C8F4632F122FC42FD0E0CC0FDD1F2C
:103A200020E2929FC00DD11D112490EA899FC00D04
:103A3000D11D1124CE0186960E942D22612FCE0128
:103A400087960E942D22DF91CF911F910895A0E0CB
:103A5000B0E0EDE2FDE10C949622A12CE12CF12CDA
:103A6000B12C00E010E0C0E0D0E06701C00ED11E34
:103A7000F601EC0FFD1FEE0FFF1FE652FB4F2591E5
:103A800034914C2F6B2D8A2D0E94001D2196C03140
:103A9000D10571F7005F1F4FB39485E0B812E3CFF3
:103AA00080E5E80EF11CA39482E0A812D9CFCDB72F
:103AB000DEB7EAE00C94B2220F931F93CF93DF930B
:103AC000823008F56530F8F44031E8F4C42FD0E0D6
:103AD000CC0FDD1F20E2629FC00DD11D112430EA02
:103AE000839FC00DD11D1124CE0186960E941F22F6
:103AF00090E0182F0027CE0187960E941F22980180
:103B0000282BC90102C080E090E0DF91CF911F9186
:103B10000F91089585E290E00E942D220895CF93A1
:103B2000C82F811102C06FEF01C062E282E290E013
:103B30000E942D22C11102C06FEF01C062E183E239
:103B400090E00E942D22C11102C06FEF01C068E019
:103B500084E290E00E942D22CF91089580E00E949F
:103B60008F1D60E070E0CB010E948A1D0E94271D1E
:103B70000E94F01C81E00E948F1D089582E290E077
:103B80000E941F22823281F483E290E00E941F2271
:103B9000823151F484E290E00E941F2291E088304B
:103BA00009F090E0892F01C080E081700895809134
:103BB000540283FF7EC087EB94E00E9471038091E2
:103BC00046021F928F9382EB94E09F938F930E9403
:103BD0000A0480EB94E00E94710380914702282F31
:103BE000082E000C330B3F938F938DEA94E09F9344
:103BF0008F930E940A048BEA94E00E9471038091E3
:103C00004802282F082E000C330B3F938F9388EA2D
:103C100094E09F938F930E940A0486EA94E00E94A6
:103C2000710380914902282F082E000C330B3F931B
:103C30008F9383EA94E09F938F930E940A0481EA12
:103C400094E00E94710380914A02282F082E000CF4
:103C5000330B3F938F938EE994E09F938F930E9451
:103C60000A048BE994E00E947103809140021F9244
:103C70008F9388E994E09F938F930E940A0486E9CA
:103C800094E00E94710380913F021F928F9383E919
:103C900094E09F938F930E940A0480E994E00E942D
:103CA00071038DB79EB74C960FB6F8949EBF0FBEAA
:103CB0008DBF0E947C1B20914702211104C02091DE
:103CC0004802222321F090934402809343022091E2
:103CD0004902211104C020914A02222321F090932D
:103CE000420280934102E0915002F09151023097DC
:103CF00049F082E0809345020480F581E02D85E45F
:103D000092E00995089580913F0280FD16C081FDE3
:103D100016C082FD18C080913E02882391F088323F
:103D200090F428E0829FC001112468E270E00E94B4
:103D30006D22862F672B29F007C082E0089584E06A
:103D4000089581E0089588E0089580913F0280FD04
:103D500014C081FD14C082FD16C0809140028823EA
:103D600081F08E3180F420E5829FC00111246EE144
:103D700070E00E946D22862F089584E1089588E204
:103D8000089588E0089580E50895CF92DF92FF922C
:103D90000F931F93CF93DF936C0100913D028091AD
:103DA0007501082BC7E0D0E010E0C8010C2E02C05E
:103DB000959587950A94E2F780FD04C02197A8F7AE
:103DC000F12C09C0FC2EB6018C2F0E940D100E9410
:103DD0001B10019799F38F2DDF91CF911F910F91B8
:103DE000FF90DF90CF900895CF93DF93EC010E9476
:103DF000C51EBE010E940D100E941B10DF91CF91C5
:103E00000895292F953078F5803168F590E030E1FC
:103E1000239F800D911D1124682F677023E09695D4
:103E200087952A95E1F7FC01EE0FFF1FE80FF91FB8
:103E3000E35AFD4F40E050E080E0219130E0062E53
:103E400002C0369527950A94E2F721703327042E95
:103E500001C0220F0A94EAF7822B4F5F5F4F433075
:103E6000510559F7089580E00895292F953088F578
:103E7000803178F590E030E1239F800D911D112471
